:1000000008308A00F7290000FF00030E8301A100D9
:100010000A08A0008A010408A2007708A300780853
:10002000A4007908A5007A08A6007B08A70083131E
:1000300083120B1E1D288B1842288C308400801ED2
:1000400023288C1A45288C308400001C29280C1881
:1000500048288C308400801C2F288C184B282208BC
:1000600084002308F7002408F8002508F900260872
:10007000FA002708FB0020088A00210E8300FF0EEB
:100080007F0E09008A110A129A298A110A12802801
:100090008A110A1268298A110A1278290A108A100C
:1000A0000A11820730342E34313400340A108A1099
:1000B0000A1182075734443454340D340A3400345E
:1000C0000A108A100A11820743344F344D344D34DC
:1000D00041344E34443420344534523452344F3455
:1000E00052340D340A34003464008C1E742818080D
:1000F000ED001A08F800ED1C7F28181218160034BD
:10010000A0307007840083130317EC010408EB0090
:100110006C10831B6C140313742003176B0884008A
:1001200083136C18831778088000A0307007840050
:1001300083130008243C031DA6280130F100F001C0
:10014000243083160313A00083120317F108031948
:1001500063297008043C031DC528043070026F3EFB
:10016000F800FA010318FA0A7808EA007A08EB00A6
:10017000A0307007840083130008EC006A08840034
:1001800083136B1883176C0880000130F007700828
:10019000063C03186329F101F00101300313EE005E
:1001A000831621082F3C0318D9282108393C03184D
:1001B000E9282108403C0318E1282108463C03189F
:1001C000E9282108603C031816292108663C031C15
:1001D000162922082F3C0318F1282208393C03185D
:1001E00001292208403C0318F9282208463C03183C
:1001F00001292208603C031816292208663C031CCA
:1002000016292208393C031807290930A2070F30A4
:10021000A2052108393C03180F290930A1070F3026
:10022000A1050310210D2204F200192983126B1677
:10023000831625082F3C031821292508393C03186B
:1002400031292508403C031829292508463C031874
:1002500031292508603C03185E292508663C031CEB
:100260005E2926082F3C031839292608393C031833
:1002700049292608403C031841292608463C031812
:1002800049292608603C03185E292608663C031CA1
:100290005E292608393C03184F290930A6070F307C
:1002A000A6052508393C031857290930A5070F3042
:1002B000A5050310250D2604F30061298312EB1612
:1002C00083168312031703138C128A110A122F2824
:1002D000D70B74290130CF070318D00A0319D10AAC
:1002E0000319D20A0F30D7000C108A110A122F28D6
:1002F000D80B84290130D3070318D40A0319D50A6F
:100300000319D60A6230D8008C108A110A122F28DD
:1003100083160C1083125208DC005108DB005008D1
:10032000DA004F08D90057080F3CE10083160C147F
:10033000831200346B1CA629EB18A629EB19A629F9
:1003400088210616831606128312EB148B108A116D
:100350000A122F288C1EAE297420AA298316861211
:10036000831286120034F415740883168700003057
:100370008312871D0130F700770D8316C700C70D64
:10038000C70DF830C7057415740887000030831254
:10039000071D0130F700F70DF70DFC30F705770862
:1003A00083164704C900F4147408870000308312D0
:1003B000871C0130F7000310F70D770883164904F6
:1003C000CB0074147408870000308312071C0130BE
:1003D00083164B048312EC00AA21EE0183168C16BF
:1003E000C03083128B048A150A12742A750884009F
:1003F00083137618831703173A088000840A800154
:10040000F50A0319F60A031300340317B91B1A2A55
:100410000F30F700380EF7050A3077020318132A59
:100420003030F707152A3908F7077708BA000313A1
:10043000F62103170F30B8050A3038020318222AB4
:100440003030242AB9133908B8073808BA00031322
:10045000F621003403173908BE003808BD003E08F5
:10046000FA003D08840083137A1883178008031963
:100470003D2ABD0A0319BE0A2F2A3B08FA003A0892
:10048000840083137A18831780080319612A3C08B3
:10049000003C0318612A3A08840083133B18831731
:1004A0000008C1003D08840083133E1883174108EB
:1004B0008000BD0A0319BE0ABA0A0319BB0ABC03AD
:1004C0003D2A3D08840083133E18831780013808B5
:1004D000F8003908F90003130034831686128312DA
:1004E000861600346D220317BA01B9013A08013C9F
:1004F000031C9A2A031D802A3908903C031C9A2A5F
:10050000F41774088316031387008312871B8D2A40
:100510000317BA01B901932A031364001030F700DE
:10052000F70B902A0317B808031D6400B90A0319D2
:10053000BA0A762A0313AA2100340C1E9D2A031737
:100540004108031399008A110A12DC2A4030840002
:10055000831700080319BD2A0130F800BF30F700E7
:100560006400F70BB02AF80BAE2A4A30F700F70BFD
:10057000B72A00006400800BAC2A003403173F1038
:1005800003136D220317BC013C08043C031CF62A2C
:1005900003136D130317BD0139083D020318E22A46
:1005A0003B08FA003A08840083133B1883170008BD
:1005B000C000C10003139D2A0317BA0A0319BB0A1E
:1005C000BD0ACC2A03136D1BEE2A03173808C0009E
:1005D0000313A62203173F14F62A03130317380840
:1005E000C0000313A6220317BC0AC42A0313AA21BE
:1005F000003003173F180130F800031300340130B6
:10060000F6001030F5003F300317BA000313F6214F
:100610006C080317B8005730B900031305222030C7
:100620000317BA000313F62101300317B900103085
:10063000B80083160313470883120317BB00831601
:100640000313460883120317BA001030BC000313CB
:100650002A2279088316C7007808C600C80148080E
:1006600046078400831347188317800803193A2B21
:10067000C80A2F2B83120317B801031372226C08C8
:100680000317B80083160313480883120317B90031
:1006900083160313470883120317BB008316031343
:1006A000460883120317BA000313BE22F808031D7D
:1006B0005F2B0A300317C0000313A6223F2B003420
:1006C0008316C70803196C2B8312EE0803196A2BD3
:1006D00083166C2B602B83168312EE08031D742B7C
:1006E0000030F800842B842B6C087202031D7F2BD2
:1006F0006B1A7F2BEE010130F800842B842B6B12D8
:10070000EE010030F800842B8A150A12E22A8316C3
:100710004708FA004608840083137A1883170008F4
:10072000CA004908FA004808840083137A1883171E
:1007300000084A02031DB32B4708FA00460884004C
:1007400083137A1883178008031DA92B0030F80043
:10075000CC2B4708FA004608C60A0319C70AC80A7C
:100760000319C90A882B4708FA0046088400831336
:10077000471883170008CA004908FA00480884008F
:1007800083134918831700084A020318CA2BFF3045
:10079000FA00CB2B0130F8008312003483160C10C2
:1007A0008312D201D101D001CF010F30D7008316BF
:1007B0000C148C108312D601D501D401D301623000
:1007C000D80083168C148312061583160611831223
:1007D0000712741274088316870083128716F412A6
:1007E00074088316870083126B148A150A12F62A7E
:1007F00020308316D200CE01CF01D001D1014908AB
:10080000FA004808F9004708F8004608F700031006
:10081000771C182C4A08CE074B0803184B0FCF073C
:100820004C0803184C0FD0074D0803184D0FD10783
:10083000D10CD00CCF0CCE0CFA0CF90CF80CF70C38
:10084000D20B072C831200348E30F70083164B082E
:10085000F8004A08F900FA01F808031D392C790854
:10086000F800F9010830F702F808031D392CF701E8
:10087000412C0310F81B402CF90DF80DF703392C0F
:10088000F8138312003483164A080319B42CD200DB
:100890004E080319B42CD2070318552C7F30D2020E
:1008A000031CB42C0319B42C592C8130D207031823
:1008B000B42C5208F700F801F901FA014B08D600F0
:1008C000D6174C08D5004D08D4001830D200D301FB
:1008D000541C822C5108FA07031C742CF90A031DBE
:1008E000742CF80A0319D3175008F907031C7B2C42
:1008F000F80A0319D3174F08CC00CC174C08F80797
:100900000318D317D30DF80CF90CFA0CD60CD50C30
:10091000D40C0310D20B672C0130F7070318B42C4A
:10092000F81B992CD60DFA0DF90DF80DF7030319E4
:10093000B42CD61FAA2CFA0A031DAA2CF90A031DEF
:10094000AA2CF80A031DAA2CF80CF90CFA0CF70AC9
:100950000319B42C4B08D3004F08D306D31FB22C75
:10096000F817B82CF813B82CF701F801F901FA01BF
:1009700083120034B630F700FA01F901F80183164A
:100980004E084F0450045104031DC82CF701D52C08
:100990000310F81BD42CCE0DCF0DD00DD10DFA0DB8
:1009A000F90DF80DF70BC82CF813831200348030C2
:1009B000831CDD2C8316D30683128316D801D9013C
:1009C0004F08D7005308D7064E080319CB2DD60081
:1009D000F70052080319D42DD6020319702D031CF9
:1009E0002E2D5308DC00DC175408DB005508DA0014
:1009F000D9010310DC0CDB0CDA0CD90CD60BF82C6B
:100A0000D71F052D5814E82D581056105816D13000
:100A100084008313FD2D5812D71B182D561C232D2F
:100A2000DC0CDB0CDA0CD90CF70A0319E32D232DAF
:100A3000DC1B262D0310D90DDA0DDB0DDC0DF703C1
:100A40000319E32D182D5817902D58134F08D70070
:100A5000D71F2C2DDC17DC2DDC13DC2D5208D60023
:100A6000F7004E08D6024F08DC00DC175008DB0008
:100A70005108DA00D9010310DC0CDB0CDA0CD90CBC
:100A8000D60B3A2DD71F472DD814E82DD810561065
:100A9000D816D53084008313FD2DD812D71B5A2DBC
:100AA000561C652DDC0CDB0CDA0CD90CF70A03198B
:100AB000E32D652DDC1B682D0310D90DDA0DDB0D40
:100AC000DC0DF7030319E32D5A2DD817902DD813F9
:100AD0005308D700D71F6E2DDC17DC2DDC13DC2D5F
:100AE0005308DC00DC175408DB005508DA00D71F78
:100AF0007D2DDC135815E82D5811D9015610D13031
:100B000084008313FD2DD71BA62D4F08D700561C3C
:100B1000902DDC0CDB0CDA0CD90CF70A0319E32D51
:100B2000D91FA12DDA0A031DA12DDB0A031DA12D5A
:100B3000DC0A031DA12DDC0CDB0CDA0CF70A03190F
:100B4000E32D581B252DD81B672DC52D8030DC06C5
:100B5000DC1FAE2DE82D5308D700BB2D4F08D70062
:100B6000DC08031DBB2DDB08031DBB2DDA08031DAC
:100B7000BB2DF701DC2DDC1BC52D0310D90DDA0DC3
:100B8000DB0DDC0DF70BBB2DE32DD71FC92DDC17BB
:100B9000DC2DDC13DC2D5208F7005308DC00540870
:100BA000DB005508DA00DC2D4E08F7004F08DC00AA
:100BB0005008DB005108DA005C08F8005B08F90017
:100BC0005A08FA001B2EF701F801F901FA011B2E51
:100BD000D901DA09DB09DC09D909D90A031DF62D87
:100BE000DA0A031DF62DDB0A0319DC0A5818042D56
:100BF000D818462D58197C2DAB2D0008DA07031C98
:100C0000072EDB0A031D072EDC0A03195614840382
:100C10000008DB07031C0F2EDC0A0319561484039B
:100C20000008801F803ADC0703185614581A0B2D51
:100C3000D81A4D2D832D8312003483164E08B63CEE
:100C4000CE00FA014F08D200CF170310CF0CD00C02
:100C5000D10CFA0CF90CF80CF70CCE0B252ED21F88
:100C60003C2EF709F809F909FA09F70A0319F80AF5
:100C70000319F90A0319FA0A83120034F701F8017B
:100C8000F901FA018316DA01DB01DC01DD01590803
:100C900058045704560403197D2E2030DE0003103B
:100CA000D20DD30DD40DD50DDA0DDB0DDC0DDD0D20
:100CB00059085D02031D662E58085C02031D662E4E
:100CC00057085B02031D662E56085A02031C772E36
:100CD0005608DA025708031C570FDB025808031C9A
:100CE000580FDC025908031C590FDD020314F70DDD
:100CF000F80DF90DFA0DDE0B4F2EDA308400831358
:100D00008312003404088316CA00C91F942ECA0334
:100D1000CA16C609C709C809C909C60A0319C70AF4
:100D20000319C80A0319C90A3B30D1009A30D00010
:100D3000CA30CF00CE010A30CC004908D50048089F
:100D4000D4004708D3004608D2005108D900500803
:100D5000D8004F08D7004E08D60083123E26000860
:100D60008316C600840A0008C700840A0008C80069
:100D7000840A0008C900F708031DD12E4C08013A67
:100D80000319D12E4A080319D32E0F394C02031927
:100D9000CB2E0318FB2ECA1BFB2E4A1BD32E203052
:100DA000F32E2030CA05CA1EE22ECA127708CA00E6
:100DB0002D3083120317BA000313F62183164A0855
:100DC000F700CA013030CA1EF32ECA127708CA00D3
:100DD0002D3083120317BA000313F62183164A0835
:100DE000F700CA013030F707770883120317BA00FB
:100DF0000313F62183165108D5005008D4004F087C
:100E0000D3004E08D200D901D801D7010A30D6004C
:100E100083123E267A088316D1007908D00078081C
:100E2000CF007708CE00CC0B9D2E831200348614A1
:100E3000831686100130F6001030F5002A30831238
:100E40000317BA000313F6216C080317B8005730D4
:100E5000B9000313052201300317B9001030B800A0
:100E600083160313470883120317BB00831603136B
:100E7000460883120317BA001030BC0003132A225D
:100E800079088316C7007808C600C80148084607D5
:100E9000840083134718831780080319512FC80A49
:100EA000462F83120317B801031372226C0803172D
:100EB000B80083160313480883120317B90083167A
:100EC0000313470883120317BB0083160313460856
:100ED00083120317BA000313BE22F808031D762FEE
:100EE0000A300317C0000313A622562F861083165C
:100EF00086108312003400306B180130F700770D34
:100F00008316C700C70DFC30C705003083126B1B6A
:100F10000130F7000310F70D770883164704C90066
:100F200000308312EB18013083164904FC00F601EF
:100F30003B30F5007C0883120317B8005730B90026
:100F4000031305220D300317BA000313F6210A30EC
:100F50000317BA000313F6218316C7013B30C600FE
:100F6000831217278A150A12182BF6013B30F50059
:100F70008316C601460883124E2000380319CA2F73
:100F80008316C60A83120317BA000313F6218316C9
:100F9000BA2F83120D300317BA000313F6210A305B
:100FA0000317BA000313F6218316C7013B30C600AE
:100FB000831217278A150A122A2BDD2F8A150A1287
:100FC0004C2B83168C1083125608E0005508DF0066
:100FD0005408DE005308DD005808623CE200831626
:0A0FE0008C1483128A150A12E62B06
:101000006B1C8428EB1C84285C088316C90083129F
:101010005B088316C80083125A088316C700831220
:1010200059088316C600CD01CC010330CB00E8304F
:10103000CA008A118312F8238A157A088316C90018
:101040007908C8007808C7007708C600CB0183126A
:1010500061088316CA008A11831224248A157A082B
:101060008316CD007908CC007808CB007708CA0039
:101070004D30D1005530D0000530CF008530CE0046
:101080008A11831243248A1577088316CA007808C8
:10109000CB007908CC007A08CD004908D100480877
:1010A000D0004708CF004608CE008A118312BA2428
:1010B0008A1583107A088316D1007908D000780841
:1010C000CF007708CE004D08D5004C08D4004B085F
:1010D000D3004A08D2008A118312D7248A157A08CD
:1010E0008316D1007908D0007808CF007708CE00A9
:1010F0008A1183121D268A157A08E6007908E50010
:101100007808E4007708E300F6013B30F500413051
:10111000840066088316C900831265088316C80018
:10112000831264088316C700831263088316C600FF
:101130008A11831282268A150D300317BA008A118C
:101140000313F6218A150A300317BA008A11031314
:10115000F6218A158316C7013B30C6008A11831217
:1011600017278A158A150A12072BF6013B30F5005E
:10117000413084006A088316C90083126908831607
:10118000C800831268088316C70083126708831695
:10119000C6008A11831282268A150D300317BA0001
:1011A0008A110313F6218A150A300317BA008A112F
:1011B0000313F6218A158316C7013B30C6008A1136
:1011C000831217278A158A150A123B2B83164608A5
:1011D0000319AC29D2004A080319AC29D202031C16
:1011E000F6287F30D2070318AC29FC288130D202C0
:1011F000031CAC290319AC295208F700F801F901C6
:10120000FA01D1014708D000D0174808CF0049089B
:10121000CE001930D2004D08CE0203181F2901302C
:10122000CF0203181F29D00203181F29D102031867
:101230001F29D10AD00ACF0A4D08CE0751294C08E0
:10124000CF0203183A290130D00203183A29D102FB
:1012500003183A29D10AD00A4C08CF074D08CE0707
:10126000031C5129CF0A031D5129D00A031D5129FE
:10127000D10A51294B088038D00203185029013077
:10128000D10203185029D10A4B088038D0074C08E6
:10129000CF07031C2E29D00A031D2E29D10A2E297F
:1012A0007A14D20B54295F290310CE0DCF0DD00D27
:1012B000D10D0310FA0DF90DF80DD30D0B29531CA8
:1012C00067290310F80CF90CFA0CD30C6A29F70300
:1012D0000319AC29D31B93290310CE0DCF0DD00DCC
:1012E000D10D4D08CE0203187F290130CF0203181B
:1012F0007F29D00203187F29D102031CA2294C08A0
:10130000CF0203188A290130D00203188A29D1029A
:10131000031CA2294B088038D002031893290130FE
:10132000D102031CA229FA0A031DA229F90A031DEE
:10133000A229F80A031DA229F70A0319AC29F80CFF
:10134000F90CFA0C4708D2004B08D206D21FAA2982
:10135000F817B029F813B029F701F801F901FA01DB
:1013600083128A150A12AE2B83164708CE004B084B
:10137000CE06CE1FC02903110310C71B0314F32987
:101380004708CE004A08CF004608CF020319CE29ED
:10139000CE1FF3290308013A8300F3294B08CF003D
:1013A0004708CF020319DA29CE1FF3290308013AAF
:1013B0008300F3294C08CF004808CF020319E6291F
:1013C000CE1FF3290308013A8300F3294D08CF000B
:1013D0004908CF020319F229CE1FF3290308013A65
:1013E0008300F329031083128A150A12E02B84016B
:1013F00083131F308305193083169900A630980097
:1014000090308312980083161F149F141F159F118C
:1014100007309C008312A901AA014630AF00B00139
:101420005130B100B2015330B300B4015630B500B1
:10143000B6014130B700B8015230B900BA01CF014E
:10144000D001D101D201D301D401D501D601D701F8
:10145000D801D901DA01DB01DC01DD01DE01DF01A8
:10146000E001E101E201E301E401E501E601E70158
:10147000E801E901EA016B10EB106B11EB116B1243
:10148000EB126B13EC01ED01F101FF30F200F301FF
:10149000F400F501F601FC01FD01FE018316BE0119
:1014A0008312EB130F30D7006230D8000C30F700F6
:1014B000073081018130840083130008F039073838
:1014C000800064000008F739F719F03977048000CC
:1014D000853090004830F80005389200FF308316C0
:1014E00092008A118312B3298A150B1683160C14E5
:1014F0008C148312071674127408831687008312E3
:101500008712F412740883168700831286108316DC
:101510008610831206118316061183120612831693
:1015200006121F1383121F179F1783169F13831210
:101530001F1483161F109F141F159F150030F800ED
:1015400083121F08C73978049F0003081839F70071
:1015500083160E08033977040E148E1483150316B0
:101560000B3A83120319B82A133A0319D92ADA2A33
:10157000F6013B30F5008316C60146088A11831236
:1015800056208A158316C60AF70083120317BA007D
:101590008A110313F6218A15053083164602031DAE
:1015A000BD2AC7013B30C6008A118312FF228A156B
:1015B000DA2ADA2A64006C088316C600C7018A1189
:1015C0008312602B8A15F80803196E2B8316C70146
:1015D0006F30C600C9012F30C8008A1183128723DB
:1015E0008A15F808031DF82A8A11CE2B8A156E2B4E
:1015F0008316C7016F30C600C9013130C8008A1197
:10160000831287238A15F808031D082B00286E2BE8
:101610008316C7016F30C600C9013330C8008A1174
:10162000831287238A15F808031D1A2B8A117B2F32
:101630008A156E2B8316C7016F30C600C90135307D
:10164000C8008A11831287238A15F808031D2C2BE2
:101650008A11B52F8A156E2B8316C7016F30C6000D
:10166000C9013730C8008A11831287238A15F80808
:10167000031D3C2BB5286E2B8316C7016F30C600A7
:10168000C9013930C8008A11831287238A15F808E6
:10169000031D4E2B8A11DD2F8A156E2BF6013B3070
:1016A000F5008316C60146088A11831260208A1548
:1016B0008316C60AF70083120317BA008A110313B0
:1016C000F6218A150F3083164602031D532BC701DE
:1016D0003B30C6008A118312FF228A156B1C852BB2
:1016E000EB18852BEB19852B8A1188218A15DC08CC
:1016F000031D842BDB08031D842BDA08031D842BB8
:1017000059081D3C0318852BEB156B1C692C6B19B4
:10171000692CEB19692C1F151F198C2B1E088316B9
:10172000CB01CA008A11831224248A157A088316F1
:10173000C5007908C4007808C3007708C2004508CE
:10174000C9004408C8004308C7004208C600CD01CC
:10175000CC01CB018730CA008312E62877088316B4
:10176000C6007808C7007908C8007A08C900CD000B
:101770004808CC004708CB004608CA00D101D00178
:101780002030CF008130CE008A11831243248A1585
:101790007A088316C5007908C4007808C300770862
:1017A000C200C901C801C7018030C6004508CD008C
:1017B0004408CC004308CB004208CA008312B42975
:1017C0000318E42B031D692C8A11E12F8A15600888
:1017D0008316C90083125F088316C80083125E084F
:1017E0008316C70083125D088316C600CD01CC01A5
:1017F0000330CB00E830CA008A118312F8238A151F
:101800007A088316C9007908C8007808C7007708E5
:10181000C600CB01831262088316CA008A118312A4
:1018200024248A157A088316CD007908CC0078081C
:10183000CB007708CA009630D1004330D000233067
:10184000CF008230CE008A11831243248A15770894
:101850008316CA007808CB007908CC007A08CD003E
:101860004908D1004808D0004708CF004608CE00FC
:101870008A118312BA248A1583107A088316D1003C
:101880007908D0007808CF007708CE004D08D50041
:101890004C08D4004B08D3004A08D2008A118312A6
:1018A000D7248A157A088316D1007908D0007808E1
:1018B000CF007708CE008A1183121D268A157A0878
:1018C000EA007908E9007808E8007708E7006B1576
:1018D0006B176B1C6F2CEB186F2CEB1D6F2CDA2A1F
:0218E0006300A3
:02400E00753FFC
:00000001FF
